:10000000A6C0B5C0B4C0B3C0B2C01FC1B0C0AFC0FD
:10001000AEC0ADC0ACC0ABC0AAC0A9C0A8C07F82F2
:1000200085888B8F9295989B9EA1A4A7AAADB0B20C
:10003000B5B8BBBEC0C3C6C8CBCDD0D2D4D7D9DB30
:10004000DDDFE1E3E5E7E9EAECEEEFF0F2F3F4F50A
:10005000F7F8F9F9FAFBFCFCFDFDFDFEFEFEFEFEE5
:10006000FEFEFDFDFDFCFCFBFAF9F9F8F7F5F4F3F3
:10007000F2F0EFEEECEAE9E7E5E3E1DFDDDBD9D72B
:10008000D4D2D0CDCBC8C6C3C0BEBBB8B5B2B0AD5C
:10009000AAA7A4A19E9B9895928F8B8885827F7C2E
:1000A0007976736F6C696663605D5A5754514E4C34
:1000B000494643403E3B383633312E2C2A272523F0
:1000C000211F1D1B1917151412100F0E0C0B0A09F6
:1000D00007060505040302020101010000000000FB
:1000E00000000101010202030405050607090A0BCD
:1000F0000C0E0F1012141517191B1D1F2123252775
:100100002A2C2E313336383B3E404346494C4E5123
:1001100054575A5D606366696C6F7376797C000032
:10012000000038000000000037000000000036002A
:10013000020202020202020202020102040810206C
:100140002004100801020000040000000000112437
:100150001FBECFE5D2E0DEBFCDBF20E0A0E6B0E01D
:1001600001C01D92A037B207E1F7BED01CC148CF35
:10017000E4E4F1E08491EAE3F1E09491E0E3F1E07A
:10018000E491EE2319F1882399F0823071F028F47C
:10019000813071F48AB58F770AC0833011F08430D2
:1001A00039F48CB58F7D8CBD03C08AB58F7D8ABD37
:1001B000F0E0EE0FFF1FE65DFE4FA591B491EC91CC
:1001C000E92381E090E021F480E0089580E090E070
:1001D0000895CF93DF9390E0FC01E65CFE4F2491FD
:1001E000FC01E05DFE4F8491882361F190E0880F6F
:1001F000991FFC01EC5DFE4FC591D491FC01E25EBC
:10020000FE4FA591B491611109C09FB7F894888100
:10021000209582238883EC912E230BC0623061F4F9
:100220009FB7F8943881822F809583238883EC913F
:100230002E2B2C939FBF06C08FB7F894E8812E2BEE
:1002400028838FBFDF91CF9108951F920F920FB631
:100250000F9211244F935F936F937F938F939F938C
:10026000AF93BF93EF93FF938091610090916200F1
:10027000A0916300B09164004091680050916900C2
:1002800060916A0070916B00840F951FA61FB71FC5
:100290008093610090936200A0936300B093640028
:1002A0008091610090916200A0916300B091640020
:1002B0008B2F9927AA27BB2780936000E0916000CD
:1002C000F0E0E25EFF4FE491E8BDFF91EF91BF9156
:1002D000AF919F918F917F916F915F914F910F900F
:1002E0000FBE0F901F901895F89420E030E080E842
:1002F0000FB6F89486BD26BD0FBE60E082E069DFD0
:1003000061E081E066DF60E080E063DF1ABC13BE7D
:1003100012BE83B7816083BF8AB580628ABD8AB509
:1003200081608ABD89B78D7F89BF80E090E0ACEDA8
:10033000B3E480936C0090936D00A0936E00B09333
:100340006F0080EA93E5AFE7B3E080936800909395
:100350006900A0936A00B0936B000ADF21E0892B4B
:1003600009F420E02093670081E080936600789490
:10037000C1E084E690E00197F1F7FADE21E0892BF5
:1003800009F420E02093670080916600281731F07F
:10039000C093650089B78D7F89BF18BC80916700C5
:0A03A00080936600E6CFF894FFCFCB
:00000001FF
